:1000000012C0189518951895189518956BC01895E5
:100010001895189518951895189518951895189578
:100020001895189518958FED8DBFC0ECE8EB4E2E06
:10003000DD275D2EEEE7F0E0A0E6B0E088278D93A7
:100040003197E9F784B7082E877F84BF8FE181BDA0
:1000500087E081BD66248FEF87BB8FEF88BB8FEF72
:1000600081BB8FEF82BB83E083BF80E080BF89B715
:10007000826089BF789480916F008F7B80936F003E
:1000800080916F008F7E80936F008FEB809367006D
:100090008FEB809368008FEB809369000027AFE6B9
:1000A0008C9187FB0EF401E041E0041709F017C0C2
:1000B00080916F008F7780936F00ACE68D919C915B
:1000C000A5E68D939C930027AFE68C9184FB0EF4FC
:1000D00001E041E0041709F001C015D17DD1DECF68
:1000E000F894FFCF0F921F922F923F924F925F9200
:1000F0007F92AF92BF920F931F932F933F934F9393
:100100005F936F937F938F939F93AF93BF93CF939F
:10011000DF93EF93FF938FB78F9385E08093520027
:10012000A2E68C918F5F8C9300916200033009F0FE
:10013000CEC080E08093620080916F0080688093E1
:100140006F00A3E68C918F5F8C930091630009315F
:1001500009F0BDC080E080936300A4E68C918F5FBE
:100160008C9300916400073009F0B1C080E0809367
:100170006400AFE68C9186FB882780F9809580FB30
:10018000AFE68C9186F98C93F89485E0E0E3F2D1A8
:100190000027AFE68C9186FB0EF401E041E00417E6
:1001A00009F011C06CEC85E0E0E3BB27A6E121E09B
:1001B0002A930CD264E485E0E0E3BB27A6E121E0CA
:1001C0002A9304D283C0002762FA0EF401E040E0D3
:1001D000041709F076C06CEC85E0E0E3BB27A6E1EC
:1001E00021E02A93F3D16EEB85E0E0E3BB27A6E1A3
:1001F00021E02A93EBD1BB27A6E185E0E0E321E0F3
:100200002A930AD2A0E65C93BB27A6E185E0E0E34F
:1002100021E02A9301D2A1E65C93A1E68C9187FBB1
:10022000AFE68C9185F98C93A1E60D91112740E002
:1002300051E059D1ACE60D931C93ACE60D911C91A5
:10024000A0E64D915527040F151FACE60D931C93A6
:100250000027AFE68C9185FB0EF401E041E0041726
:1002600009F00DC0ACE642E0F7D0ACE60D911C9170
:1002700041E050E0040F151FACE60D931C93ACE673
:100280000D911C914AE050E02ED1ACE60D931C93E9
:10029000ACE60D911C9140E150E00BD1ACE64D93E2
:1002A0005C930027AFE68C9184FB0EF401E040E004
:1002B000041709F005C080916F00806180936F0082
:1002C00005C080E197E2ACE68D939C9378948F9182
:1002D0008FBFFF91EF91DF91CF91BF91AF919F9130
:1002E0008F917F916F915F914F913F912F911F91CE
:1002F0000F91BF90AF907F905F904F903F902F9065
:100300001F900F901895A5E60D911C91083E53E0A3
:10031000150708F057C0A5E60D911C914AE050E082
:10032000C8D0AAE60D931C9380916A008093670061
:10033000A5E60D911C914AE050E0BBD0A5E64D9397
:100340005C93A5E60D911C914AE050E0B2D0AAE67C
:100350000D931C9380916A0080936800A5E60D912F
:100360001C914AE050E0A5D0A5E64D935C93A5E62C
:100370000D911C914AE050E09CD0AAE60D931C938D
:1003800080916A008093690000916900003009F053
:1003900003C08AE080936900E0E4F4E0A7E68C9172
:1003A0009927A7E6CCD0ECE4F4E0A8E68C91992755
:1003B000A8E6C5D0E0E4F4E0A9E68C919927A9E687
:1003C000BED009C08FEA809367008FEA80936800EF
:1003D00086E8809369000895AEE68C918F5F8C93D8
:1003E00000916E00033009F003C080E080936E003E
:1003F000AFE68C9185FB882780F9809580FBA2E38E
:100400008C9186F98C9300916E00003009F006C043
:10041000909AA9E68C9188BB929811C0013009F09E
:1004200006C0929AA8E68C9188BB919808C00230C9
:1004300009F005C0919AA7E68C9188BB9098089521
:10044000C0F9A4B0999282F88090FF0040792430DE
:10045000191202780010FF00EA2FFB2F8D91809572
:1004600081934A95D9F7089508D03DD000FC10D06B
:10047000089503D01ED001F8F9CF0024E89457FF67
:1004800002C009D0689400F80BD010F80124089538
:1004900002D009D00895509540954F5F5F4F089561
:1004A000E89417FF0895009510950F5F1F4F68940B
:1004B0000895352F242FE894452B11F4689408955E
:1004C000512F402F0027112780E1440F551F001F97
:1004D000111F021B130B416018F4020F131F4E7FF4
:1004E0008A9599F70895752F642F55274427FF9310
:1004F000F1E1889405C010F4460F571F56954795B3
:1005000017950795FA95B9F7FF9108953197F1F787
:100510000895689462F80895E89462F80895C8957B
:1005200031960020089591E005C092E003C094E068
:1005300001C098E0F4DF0D929A95E1F70895E80F75
:10054000F91FF1CF91E0882321F08894991F8A95B3
:10055000E9F7892F909508950181082B0183128175
:1005600019231283EF93FF93E2E0F0E0CFDFFF91D6
:10057000EF910895CEDFFF27E5DFEEDFEF93FF93E6
:10058000ECE9F5E0C3DFFF91EF91182B128309230B
:100590000183EF93FF93EAE0F1E0B8DFFF91EF9181
:1005A0001081182359F4EF93FF93ECE9F5E0AEDFE7
:1005B000FF91EF911081182309F0AEDFEF93FF93C5
:1005C000ECE9F5E0A3DFFF91EF910895BBDFFF2792
:1005D00029915D9148E0C0DFEF93FF93E2E0F0E006
:1005E00095DFFF91EF91579510F4182B1283EF933D
:1005F000FF93E0EBF0E08ADFFF91EF91182B12837D
:10060000EF93FF93E2E0F0E081DFFF91EF914A95F5
:1006100011F72A95F1F6089595DFFF27299148E013
:1006200055279ADF09230183EF93FF93EEE0F0E073
:100630006DDFFF91EF9188941081182309F00894E1
:100640005795EF93FF93E3E8F0E060DFFF91EF91C0
:0C0650004A9539F75D932A9511F708953B
:00000001FF
